:1000000008308A00D5280000FF00030E8301A100FC
:100010000A08A0008A010408A2007708A300780853
:10002000A4007908A5007A08A6007B08A70083131E
:1000300083128C308400801E1F288C1A3C288C3040
:100040008400801C25288C183F288B1E29280B191A
:100050004228220884002308F7002408F800250815
:10006000F9002608FA002708FB0020088A00210E64
:100070008300FF0E7F0E09008A110A12C12A8A111D
:100080000A12BC2A8A110A12E7290A108A100A11D8
:10009000820728340C34013406340A108A100A11FD
:1000A00082070C344F3476346534723400340A10CD
:1000B0008A100A1182070C344634493446344F34CE
:1000C00000340A108A100A118207303400340A10F2
:1000D0008A100A118207BA346934BC3420340034DF
:1000E0000A108A100A118207A8346F34BD346534AF
:1000F000E3346934BB346F34BA3400340A108A10E4
:100100000A11820742346934B334BF346F34703417
:100110006F34BA3400340A108A100A11820743344B
:10012000653470346534E334613400340A108A1065
:100130000A118207AB346534BF34B334653470348C
:1001400000340A108A100A118207A8342734C734F1
:10015000BF34BD34B834E534C73400340A108A10D3
:100160000A1182073A3400340A108A100A118207F1
:100170002E3400340A108A100A118207433479346D
:10018000B2346F34BF34613400340A108A100A115B
:10019000820748346534E3346934BB34C7340034EF
:1001A0000A108A100A118207203400340A108A10BB
:1001B0000A1182070C3444344934533450344C34DB
:1001C000413459342034763431342E3430340A34C6
:1001D0006234753469346C346434203433343134EB
:1001E00020342834303434342E34303435342E3402
:1001F00030343934293400340A148A100A11820741
:100200000C3400340A148A100A1182070C34453465
:10021000723472343A340034F0308316880083121A
:1002200008150000081400000808080E0F3983168E
:1002300003179E00831203130810000008146400C3
:100240000808080E0F39831603179D008312031345
:10025000081000308316880003171E0EF700F030D8
:10026000F70577081D04F800831203130034831682
:1002700003171E0EF039F7000F3083120313080521
:10028000770488000000081464000000081000349F
:1002900088100C217808831603179D009D1F532991
:1002A0008312031349291B185A2983120313881038
:1002B000831603171B1C61298312031388148316EA
:1002C000031700008312031308110000081083169F
:1002D00003171C0E9D000F309D051D089E00831204
:1002E00003133721831603171C080F399D009E0046
:1002F00083120313372100349730840083170008DA
:10030000031993290130F800BF30F7006400F70BA0
:100310008629F80B84294A30F700F70B8D29000055
:100320006400800B8229003483160317180B992967
:100330009C29403099009D299901013017029907A5
:10034000190880389A009B011A089C008312031335
:10035000482100348316031716080C3A831203133E
:100360000319B929063A0319C929023A0319D329ED
:10037000DC29831603179B0101309C0083120313B1
:1003800048210230831603179700831203137C2140
:10039000E629013083160317970002309800831274
:1003A00003139421E629831603179B0110309C0048
:1003B000831203134821E6290130831603179B009B
:1003C00016089C00831203134821E6290034981C68
:1003D000002A8316031795011508831203134D2075
:1003E00000380319FF2983160317950A9600831214
:1003F0000313AA2183160317EC2983120313FF2981
:10040000420B192A8316031795011508831203134B
:10041000572000380319182A83160317950A9600E7
:1004200083120313AA2183160317052A83120313C9
:10043000182AB10A31080F3C0318B42AB00AB101D6
:1004400030083B3C0318B42AB001AF0A2F083B3CEC
:1004500003182C2AAE0AAF012E08173C0318B42A41
:10046000AD0AAE012D081C3C031C382A0030392A85
:100470000130831603179500831203132C08023CE6
:100480000319442A0030452A013083160317150545
:100490000319502A83120313AD01AC0A8316031704
:1004A000831203132D081E3C031C582A0030592ABE
:1004B0000130831603179500831203132C08043CA4
:1004C0000319642A0030652A013083160317960049
:1004D000831203132C08063C0319702A0030712A7A
:1004E00001308316031716059700831203132C0897
:1004F000043C03197D2A00307E2A0130831603173D
:1005000017059800831203132C08093C03198A2A43
:1005100000308B2A013083160317180599008312C7
:1005200003132C080B3C0319972A0030982A01303A
:1005300083160317190515050319A42A831203133B
:10054000AD01AC0A83160317831203132D081F3C59
:100550000318AC2AAD01AC0A2C080C3C0318B42AD1
:10056000AA0A0319AB0AAC013A08F93C0318BA0A03
:100570000B118A110A122928B40A8C108A110A1246
:1005800029281A08831603179500831203134108BC
:100590001E3C031CDE2A433040078400831383166D
:1005A00003171508800083120313C00AC10A40080C
:1005B0001E3C0318DC2AC0016400E02A0130C2009E
:1005C0008C128A110A122928C108031DE92A640025
:1005D000E42AC1080319FC2A43303F07840083132F
:1005E00000080317EA000313C103BF0A3F081E3CBB
:1005F0000318FB2ABF01640003176A08F8000313FD
:1006000000340C1E012B0317540803139900003407
:1006100002300317D4000313012303175308D40037
:10062000031301230034AB01AA01E422FA01780884
:10063000AA047A08AB04E4220317D2017808D10097
:10064000FA0000300313AA047A08AB04153003172C
:10065000D300031308238A150A123C2C0317D10177
:1006600051080313FC2000380319482B0317D10A43
:100670000313A8018B1BA8178B138316031796006F
:1006800083120313AA21A81B8B170317302B031304
:1006900020300317D300031308238A150A12AE2D46
:1006A00007100317EC01EF016C08073C031CB02B8B
:1006B00003130618602BB408031D602B6400592B2C
:1006C000061C672BB408031D672B6400602B0618FB
:1006D0006E2BB408031D6E2B6400672B11080317E3
:1006E000ED0003133408013C0318792B0317B02BDA
:1006F0000313B4013408910003176D08393C031843
:10070000832B0030842B01308316900083126D08F8
:10071000AE3C031C8D2B00308E2B01308316100451
:100720000319992B013083120313B4000317B02B64
:10073000831683126D08633C0318EE016D08743C48
:100740000318AE2B0130EE006C08F8000319AC2B37
:100750000310EE0DF80BA82B6E08EF04EC0A542BD7
:100760000313390BB72B03176F080313B5003908B0
:10077000023C031DBF2B03176F080313B600390893
:10078000033C031DC72B03176F080313B700390879
:10079000043C031DCF2B03176F080313B800031786
:1007A0006F08EB000313B408031DDA2B0130F800C7
:1007B000DD2BDD2B0030F800DD2B00343C0BE12B72
:1007C000622C0317EA016A080313B800B700B600E9
:1007D000B5000030F80005389200FF308316920013
:1007E0008C148312B401340891000618FD2B3408D0
:1007F0000A3C031CFD2B6400F52B34080A3C031C47
:100800005C2CB401340891003408023C031C0A2C0F
:100810006400042C0030F80006389200FF30831684
:1008200092008312B40134089100003006180130A0
:100830000317EC000313B4080319202C0030212CFB
:10084000013003176C050319292C64000313152CC0
:1008500003170313B408031D5C2CB4013408910082
:100860000130B90035080317EB0003135023F808D3
:1008700003195C2C0230B90036080317EB00031390
:100880005023F80803195C2C0330B900370803170C
:10089000EB0003135023F80803195C2C0430B90053
:1008A00038080317EB0003135023F80803195C2CD6
:1008B00083168C108312622CBC0185100030F80066
:1008C000672C672C0130BC008514F800672C0034BD
:1008D00094138C1103175808031393000230941BD0
:1008E000782C8C1D712C00308316111B0130831263
:1008F000F8000034E4227808313C031D062DE42280
:100900007808393C031DFE2C831611141118862C0F
:10091000A63083120317D800031368246400103034
:10092000F700F70B912C0317D80103136824031762
:10093000D801031368240317D301D20183160313CC
:1009400091149118A12C64002030F700F70BA62C0D
:10095000A92CA63083120317D8000313682464005F
:100960002030F700F70BB22CB52C03175308D40036
:10097000D5015308D8000313682464002030F70021
:10098000F70BC02CC32C03175208D800031368249C
:10099000E42278080317D1005108D8000313682413
:1009A0000317D108031DD92C5108D800031368245C
:1009B000031764002030F700F70BDC2CDF2C8316C4
:1009C000031311151119E22C8312A8018B1BA81710
:1009D0008B130630831603179700831203137C21B1
:1009E000A81B8B1764000317D20A0319D30AD10876
:1009F0000319FC2C510F9E2C042D0313FF300317F9
:100A0000D4000313012303170C2D0313FF30031726
:100A1000D40003130123031703138A150A12902D20
:100A20006C08840083136D1883170317690880000E
:100A3000840A80010313EC0A0319ED0A003403173A
:100A4000D20152080313022100380319392D03176C
:100A5000D20A0313A8018B1BA8178B138316031745
:100A6000960083120313AA21A81B8B170317212DAD
:100A700003130317D6015108D500D701D801D901B6
:100A8000DA01DB01DC01DD01DE0101300313ED00E1
:100A90005730EC001030840003175608E100550869
:100AA000E000E8010408E7006810831B6814610E89
:100AB000F038E300E307E23EE400323EE60061087E
:100AC0000F39E407E407E607E93EE500E507E50737
:100AD000600E0F39E507E607E50DE60DE609E60DC0
:100AE00060080F39E607E30D0730E2000A30E60739
:100AF000E503031C772DE507E403031C7B2DE407C6
:100B0000E303031C7F2DE307E203031C832D623004
:100B10008400831707306705671384076630040273
:100B2000031967170008F700031D9E2D671B9E2DF4
:100B3000671AB22DE7199E2D2030A12DE7156712F7
:100B40003030F707E1010408E0006110831B6114F5
:100B50007708E90003131025031760088400831346
:100B600061188317840A671F8E2DDF015F08073C19
:100B7000031CDA2D57305F07840083170008203CE0
:100B80000318D72D57305F07840083170008E00053
:100B90000313A8018B1BA8178B1303176008831678
:100BA000960083120313AA21A81B8B170317DF0AD1
:100BB0006400B62D03138A150A12AE2D03175F08C1
:100BC000F8015E020318E72D5E08F700F32DF70128
:100BD0000830E000DE0DF70D5F0877020318F7001C
:100BE000F80DE00BEA2D031300340130ED00553011
:100BF000EC0003175408D8001130D9002030591EDA
:100C00003030DA005808F700D81F0D2EF709F70A20
:100C10007708D8002D30DA00D9175808DE00643084
:100C2000DF000313DE2577080317D800303078077C
:100C3000DB005808DE000A30DF000313DE25303009
:100C400077070317DD0030307807DC005A08F7001B
:100C5000D91D2C2ED91F5911591A392ED91F542E8E
:100C60005919542E7708DB00D918542E7708DC0068
:100C7000542E30305B02031D542E7708DB002030E9
:100C8000DA00D91D472E5911D914D91FD910303087
:100C90005C02031D542E7708DC002030DB00D91DD8
:100CA000472ED910D91F5910591D5B2E5A08E9003B
:100CB000031310250317D91C622E5B08E9000313E8
:100CC00010250317591C692E5C08E9000313102531
:100CD00003175D08E9000313102503175508203C8E
:100CE000031D742E3030D50030305502F700770EDA
:100CF000D700F030D70530305602D7075708F80034
:100D00000313003405128316051264005230F700F5
:100D1000F70B882E8B2E64004C30F700F70B8E2ECD
:100D2000051664000430F700F70B942E00008312C0
:100D300003175110D2015208243C031CA82ED20ADA
:100D40000313051AA62E03175114031303179B2E22
:100D50006400003051180130F80003130034031709
:100D6000D2015208073C031CD62E51080139013C20
:100D7000031DC72E831603130512640005166400B5
:100D80001A30F700F70BC22ED02E831203178316EA
:100D90000313051264001A30F700F70BCD2E051669
:100DA000031083120317D10CD20AB12E640003136F
:100DB0000034E408031DDE2EE508031D502F0B133D
:100DC0008B138B1BE02E8226780B4E2F6400CC30C9
:100DD0000317D1000313AF2664002030F700F70B90
:100DE000EF2EF22EBE300317D1000313AF2664009E
:100DF0002030F700F70BFA2EFD2E0317D101510812
:100E0000073C031C3C2F0130FF000310D20C83165B
:100E1000031305126400051664000E2F00008312F0
:100E2000051EFF01051EFF01051EFF01051EFF0136
:100E3000051EFF01051EFF01051EFF01051EFF0126
:100E4000051EFF01051EFF01051EFF01051EFF0116
:100E5000051EFF01051EFF01051EFF017F0B332F3D
:100E60000317D217031364000430F700F70B362F73
:100E700000000317D10AFF2E64005208F80078081A
:100E80000313EA008226CC300317D1000313AF26E8
:100E9000640044300317D1000313AF26C0308B0425
:100EA000E40A0319E50A8A150A125A2E83169115C7
:100EB0009119582F77189112771C91161116111A43
:100EC0005F2F83121308F80000348E30F7000317E9
:100ED0005308F8005208F900FA01F808031D7A2FA8
:100EE0007908F800F9010830F702F808031D7A2F95
:100EF000F701822F0310F81B812FF90DF80DF7036E
:100F00007A2FF8130313003403175308DA00570835
:100F1000DA06DA1F902F03110310D31B0314C32F1B
:100F20005308DA005608DB005208DB0203199E2F33
:100F3000DA1FC32F0308013A8300C32F5708DB00D1
:100F40005308DB020319AA2FDA1FC32F0308013A43
:100F50008300C32F5808DB005408DB020319B62FA7
:100F6000DA1FC32F0308013A8300C32F5908DB009F
:100F70005508DB020319C22FDA1FC32F0308013AF9
:100F80008300C32F0310031300340317D201520848
:100F90000313702000380319DF2F0317D20A03133D
:100FA000A8018B1BA8178B138316031796008312B7
:100FB0000313AA21A81B8B170317C72F03138A112A
:100FC0000A16ED2C0317D201520803137E200038B5
:100FD0000319FC2F0317D20A0313A8018B1BA817B0
:100FE0008B1383160317960083120313AA21A81BE1
:0E0FF0008B170317E42F03138A110A16F42C33
:101000000317D20152088A1103138B208A15003866
:1010100003191E280317D20A0313A8018B1BA81754
:101020008B138316031796008A1183120313AA21C8
:101030008A15A81B8B170317022803138A110A1697
:10104000FC2C0317D20152088A11031396208A152B
:10105000003803193F280317D20A0313A8018B1B7A
:10106000A8178B138316031796008A118312031394
:10107000AA218A15A81B8B170317232803138A118B
:101080000A16052D0317D20152088A110313A12055
:101090008A150038031960280317D20A0313A80120
:1010A0008B1BA8178B138316031796008A118312C4
:1010B0000313AA218A15A81B8B17031744280313AF
:1010C0008A110A160E2DF701F80103175A080310AA
:1010D0005B18F707F70CF80CDB18F707F70CF80CA0
:1010E0005B19F707F70CF80CDB19F707F70CF80C8E
:1010F0005B1AF707F70CF80CDB1AF707F70CF80C7C
:101100005B1BF707F70CF80CDB1BF707F70CF80C69
:10111000031300343508023C03199A283608FD3CB5
:1011200003199A283608033C03199A283608FC3C10
:10113000031DD2283808FF3C3702031DD228370888
:101140003B02031DA7283A08063C0318D2280330A7
:101150000317D4008A11031301238A153508023CB2
:101160000319B6283608FD3C031DBD2837080317B0
:10117000D4008A11031301238A153508033C03198F
:10118000C5283608FC3C031DCE28E030370703177E
:10119000D100D4008A11031301238A15BA0137083C
:1011A000BB0085108A150A129C2F840183131F30FF
:1011B0008305A91529088316870083122916290893
:1011C0008316870009309300283083129400831619
:1011D0009417141303170908C039890003131F1249
:1011E0009F1200300317880083128701880189014C
:1011F000FF300313A9000E30031790001130910047
:10120000103092001C309300103094001130950083
:101210000E3096009701980199019A0010309B00BA
:101220001C309C0010309D000E309E009F010A3043
:10123000A000A1010430A200A300A400A5000E306C
:10124000A600A7010A30A800A9010C30AA000430AA
:10125000AB00AC00AD000E30AE00AF010230B0000C
:101260000530B1000230B200B301B401B501B601DE
:10127000B701B801B9011E30BA000830BB00043014
:10128000BC000830BD001E30BE00BF011F30C000D2
:10129000C101C200C301C400C501C600C701C80026
:1012A000C901CA00CB01CC00CD01CE00CF01031390
:1012B000EC01ED010730AB00D830AA00B2013208D2
:1012C000B000AF00AE00AD00AC000130B300AF30F5
:1012D000831685009E30870000308800003088002B
:1012E0008312881008110810A8018B1BA8178B13F4
:1012F0000F308316031797008A11831203137C2182
:101300008A15A81B8B1701300317D2005208033C23
:10131000031CAC290313A8018B1BA8178B130330E4
:10132000831603179E008A118312031337218A152F
:10133000A81B8B17A8018B1BA8178B1305308316CE
:10134000031797008A11831203137C218A15A81BA7
:101350008B170317D20A86290313A8018B1BA81722
:101360008B130230831603179E008A118312031316
:1013700037218A15A81B8B170317D2015208033C8B
:10138000031CDF2952088A11031345208A1503170D
:10139000D3000313A8018B1BA8178B138316031705
:1013A0009B018312530883169C008A118312031336
:1013B00048218A15A81B8B170317D20ABE290313CD
:1013C000A8018B1BA8178B13831603179B014030B2
:1013D0009C008A118312031348218A15A81B8B17BE
:1013E00064000E30F700F70BF32900000317D20159
:1013F00052083F3C031C1E2A1030520784008317FA
:101400000008D3000313A8018B1BA8178B1301300E
:10141000831603179B008312530883169C008A11BE
:101420008312031348218A15A81B8B176400103000
:10143000F700F70B192A0317D20AF8290313A8019A
:101440008B1BA8178B13831603179B0180309C00FE
:101450008A118312031348218A15A81B8B17831640
:1014600003170908C039890003131F129F120030A7
:1014700003178800831203131F101730031785000A
:10148000831603130108F039810064000108C03994
:1014900007388100831290015830F8000638920016
:1014A000FF30831692008312031787018801890198
:1014B00083160313970183120317D20152088A116E
:1014C0000313D6208A15003803197A2A0317D20A83
:1014D0000313A8018B1BA8178B1383160317960001
:1014E0008A1183120313AA218A15A81B8B170317CD
:1014F0005E2A0313A8018B1BA8178B13FF308316DA
:10150000031797008A11831203137C218A15A81BE5
:101510008B17A8018B1BA8178B13FF30831603179B
:1015200097008A11831203137C218A15A81B8B173D
:10153000A8018B1BA8178B13FF3083160317970086
:101540008A11831203137C218A15A81B8B17A8010B
:101550008B1BA8178B13FF308316031797008A1174
:10156000831203137C218A15A81B8B17A8018B1BE0
:10157000A8178B13FF308316031797008A11831265
:1015800003137C218A15A81B8B17A8018B1BA81796
:101590008B13FF308316031797008A1183120313EE
:1015A0007C218A15A81B8B17A8018B1BA8178B13EE
:1015B000FF308316031797008A11831203137C21CF
:1015C0008A15A81B8B170317D1015108183C031C5F
:1015D000F02AA0305107840083138001D10AE52A44
:1015E00001300313BE001930831699001812181326
:1015F00018158C1683121813181698178316981638
:101600008312C0014008C100BF00C100C2008B1698
:10161000BC010317D20152088A110313FC208A155A
:1016200000380319272B0317D20A0313A8018B1BB9
:10163000A8178B138316031796008A1183120313BE
:10164000AA218A15A81B8B1703170B2B0313640001
:10165000C0308B04C1080319352B8A11E4228A1586
:1016600078080317D000372B03130317D001500855
:10167000031303197B2B013A03197C2B043A03193A
:10168000842B033A0319942B013A0319B42B0D3A16
:101690000319BF2B1A3A0319CE2B013A0319E02B79
:1016A000033A0319F22B013A0319042C073A0319E0
:1016B000162C213A0319282C203A03193A2C353AD2
:1016C0000319432C013A0319462C033A0319772CCA
:1016D000013A0319AE2CA33A03190F2D013A03194D
:1016E0002C2D033A0319482D013A0319642DB33AFE
:1016F00003198E2D992DAE2D01300317D3008A11B9
:10170000031308238A15AE2DFF300317D4008A1166
:10171000031301238A1503175008D4008A110313F9
:1017200001238A15B301AE2D06300317D1005108ED
:10173000053C031D9E2B0313B30103175108063C00
:10174000031DA62B01300313B30003178A110313E3
:10175000E4228A1578080317D2005108D3008A11B1
:10176000031308238A15AE2D8A11E4228A15073047
:101770000317D3008A11031308238A15AE2DFF30F7
:101780000317D4008A11031301238A150317500885
:10179000D4008A11031301238A15AE2D8A11E42285
:1017A0008A157808AE0010300317D3008A1103138E
:1017B00008238A150330BE00E3013E08E200AE2D87
:1017C0008A11E4228A157808AF0011300317D3007C
:1017D0008A11031308238A150330BE00E3013E0873
:1017E000E200AE2D8A11E4228A157808B00012308A
:1017F0000317D3008A11031308238A150330BE0090
:10180000E3013E08E200AE2D8A11E4228A15780831
:10181000AD0013300317D3008A11031308238A1570
:101820000330BE00E3013E08E200AE2D8A11E4223F
:101830008A157808AC0014300317D3008A110313FB
:1018400008238A150330BE00E3013E08E200AE2DF6
:101850008A11E4228A157808B20035300317D300C4
:101860008A11031308238A150330BE00E3013E08E2
:10187000E200AE2D8A11132B8A150330BE00E3015E
:101880003E08E200AE2D8A112E2B8A150317D201D5
:1018900052083F3C031C502C5208D300D401552C55
:1018A00040305202D3000130D40001305307D5003C
:1018B00001305407D6000313A8018B1BA8178B1304
:1018C000031755088316970083125608831698004D
:1018D0008A118312031394218A15A81B8B172130B8
:1018E0000317D3008A11031308238A15AE2D8A111A
:1018F000E4228A1578080317D1005108D200520853
:101900003F3C031C872C5208D300D4018C2C403060
:101910005202D3000130D40001305307D50001300A
:101920005407D6000313A8018B1BA8178B130317AA
:1019300055088316970083125608831698008A115B
:101940008312031394218A15A81B8B1722300317C7
:10195000D3008A11031308238A15AE2D0317D20171
:101960005208143C031CBB2C5430520784008317CC
:101970008001D20AB02C8A110313E4228A15780858
:101980000317D100D201D1080319DA2C54305207C1
:1019900084008317510880008A110313E4228A15FA
:1019A00078080317D100D20A5208153C031CDA2C20
:1019B0006400C32CD301520853020318072D54307E
:1019C00053078400831780080319FD2C54305307F4
:1019D000840083170008EA000313A8018B1BA817D3
:1019E0008B1303176A08831696008A118312031358
:1019F000AA218A15A81B8B17031703130618032D9A
:101A00008A11DE238A1564000317D30ADB2C2330E6
:101A1000D3008A11031308238A15B301AE2D803039
:101A20000317D3008A11031308238A158030031784
:101A3000D4008A11031301238A1555300317D400EB
:101A40008A11031301238A15AA300317D4008A11BF
:101A5000031301238A15AE2D81300317D3008A1199
:101A6000031308238A1581300317D4008A11031346
:101A700001238A1501300317D4008A1103130123AF
:101A80008A150317D4018A11031301238A15AE2D79
:101A900082300317D3008A11031308238A1582307A
:101AA0000317D4008A11031301238A150230031788
:101AB000D4008A11031301238A150317D4018A1154
:101AC000031301238A15AE2D83300317D3008A1127
:101AD000031308238A1583300317D4008A110313D4
:101AE00001238A1533300317D4008A11031301230D
:101AF0008A1534300317D4008A11031301238A1581
:101B000035300317D4008A11031301238A150317F4
:101B1000D4018A11031301238A15AE2D8A117A2C60
:101B20008A1530300317D3008A11031308238A154E
:101B3000AE2DFF300317D4008A11031301238A1539
:101B400003175008D4008A11031301238A150317C1
:101B50005008D1008A1103131F2D8A156400031742
:101B60005008123C031D482E83160313111411183C
:101B7000B72DD03083120317D8008A1103136824BD
:101B80008A150317D8018A11031368248A153008AF
:101B90000317D4008A110313F5258A157808031753
:101BA000D1005108D8008A11031368248A152F0820
:101BB0000317D4008A110313F5258A157808031733
:101BC000D1005108D8008A11031368248A152E0801
:101BD0000317D4008A110313F5258A157808031713
:101BE000D1005108D8008A11031368248A153208DD
:101BF0000317D8008A11031368248A152D080317C8
:101C0000D4008A110313F5258A1578080317D1002B
:101C10005108D8008A11031368248A152C08031769
:101C2000D4008A110313F5258A1578080317D1000B
:101C30005108D8008A11031368248A15D0302A026B
:101C40000317D20003132B080317D3000730031C1C
:101C50000830D3025208D4008A110313F5258A15DF
:101C600078080317D1005108D8008A11031368249B
:101C70008A150317D1015108D8008A11031368246B
:101C80008A15831611151119432E64008312031748
:101C9000031306184E2E8A11DE238A150317D00867
:101CA000031D8E2F0313330B562E582E03178E2F22
:101CB0008A11D92E8A1569081F3C0318842FE9015F
:101CC000E8010B138B138B1B622E8316A008031DD8
:101CD0006D2E8312E701E601831683120317D101EB
:101CE0005108173C031C8E2EA0305107F800FA0152
:101CF0000318FA0A7808D2007A08D3000130510795
:101D0000A03E840083130008D5005208840083138A
:101D10005318831755088000D10A702E83160313B9
:101D2000B801640083120317D101A0305107840069
:101D3000831380080319A22E5108183C031CA22EFD
:101D4000D10A952E5108133C031C482F64001D3006
:101D5000F700F70BA92E00008316031311141118B6
:101D6000AF2EA73083120317D8008A1103136824FB
:101D70008A1503175108183C031C3E2F6400543089
:101D8000F700F70BC12E000064005108173C031C3C
:101D9000D72EA0305107840083130130F7008A1139
:101DA000031356278A1578088000E22E0317A03007
:101DB000510784008313F7018A11031356278A15EC
:101DC00078088000A030031751078400831380082F
:101DD000031D372FF7018A11031356278A1583161F
:101DE00011151119F12E11141118F42EA6308312A9
:101DF0000317D8008A11031368248A150317D80122
:101E00008A11031368248A150317D8018A11031352
:101E100068248A158316911491180C2FA730831209
:101E20000317D8008A11031368248A150317510871
:101E3000173C031C292FA030510784008313013065
:101E4000F7008A11031356278A1578088000342F6B
:101E50000317A030510784008313F7018A1103137D
:101E600056278A1578088000E701E6010317D10A92
:101E70000313E60A0319E70AB92E0317831603139F
:101E800011151119412F11151119442F8312031720
:101E9000D1010313A8018B1BA8178B1301308316E4
:101EA00003179700023098008A11831203139421BC
:101EB0008A15A81B8B1703175108133C031C812F8D
:101EC000A030510784008313800803197E2FA030AF
:101ED0005107840083130008D2000313A8018B1B51
:101EE000A8178B1303175208831696008A118312C2
:101EF0000313AA218A15A81B8B170317D10A6400A4
:101F00005C2FC03003138B04E80A0319E90A0A1690
:101F10008A1100280A128A156400031703133C0B68
:101F20009D2FC108031D9D2F0317D00803199A2F59
:0E1F300003139D2F03138A28BC012A2B630084
:10200000BD0AC108031DCE2F330BCE2F3D08FA3C6D
:102010000318CE2FA8018B1BA8178B130130831632
:102020000317970098000A128312031394210A16CB
:10203000A81B8B17C108031DE7282E08093C031CA9
:102040003F280317D20152080A12031361200A160F
:10205000003803193F280317D20A0313A8018B1B6A
:10206000A8178B138316031796000A128312031303
:10207000AA210A16A81B8B1703172328031303177B
:10208000D60103132E080317D500D701D801D901B3
:10209000DA01DB01DC01DD01DE0101300313ED00BB
:1020A0005730EC001030840003175608E100550843
:1020B000E000E8010408E7006810831B6814610E63
:1020C000F038E300E307E23EE400323EE600610858
:1020D0000F39E407E407E607E93EE500E507E50711
:1020E000600E0F39E507E607E50DE60DE609E60D9A
:1020F00060080F39E607E30D0730E2000A30E60713
:10210000E503031C7F28E507E403031C8328E40799
:10211000E303031C8728E307E203031C8B286230D8
:10212000840083170730670567138407663004024D
:10213000031967170008F700031DA628671BA628C8
:10214000671ABC28E719A6282030A928E7156712C6
:102150003030F707E1010408E0006110831B6114CF
:102160007708E9000A12031310250A1603176008FE
:102170008400831361188317840A671F9628DF0180
:102180005F08073C031CE62857305F07840083176D
:102190000008203C0318E32857305F0784008317AA
:1021A0000008E0000313A8018B1BA8178B1303176B
:1021B0006008831696000A1283120313AA210A16D6
:1021C000A81B8B170317DF0A6400C0280313C1087C
:1021D000031D08290317D20152080A120313AE2067
:1021E0000A160038031908290317D20A0313A80195
:1021F0008B1BA8178B138316031796000A128312E2
:102200000313AA210A16A81B8B170317EC28031324
:10221000C108031DD5292F08093C031C2D290317CC
:10222000D20152080A12031361200A16003803195A
:102230002D290317D20A0313A8018B1BA8178B1390
:102240008316031796000A1283120313AA210A1693
:10225000A81B8B170317112903130317D6010313A8
:102260002F080317D500D701D801D901DA01DB0106
:10227000DC01DD01DE0101300313ED005730EC001D
:102280001030840003175608E1005508E000E8010B
:102290000408E7006810831B6814610EF038E3003F
:1022A000E307E23EE400323EE60061080F39E4074E
:1022B000E407E607E93EE500E507E507600E0F39AC
:1022C000E507E607E50DE60DE609E60D60080F39BE
:1022D000E607E30D0730E2000A30E607E503031CDA
:1022E0006D29E507E403031C7129E407E303031CDC
:1022F0007529E307E203031C792962308400831700
:1023000007306705671384076630040203196717EF
:102310000008F700031D9429671B9429671AAA294E
:10232000E719942920309729E71567123030F7070D
:10233000E1010408E0006110831B61147708E900E3
:102340000A12031310250A1603176008840083136A
:1023500061188317840A671F8429DF015F08073C1F
:10236000031CD42957305F07840083170008203CE2
:102370000318D12957305F07840083170008E00055
:102380000313A8018B1BA8178B1303176008831670
:1023900096000A1283120313AA210A16A81B8B1790
:1023A0000317DF0A6400AE290313E20A0319E30AE4
:1023B000A8018B1BA8178B130730831603179700F0
:1023C000013098000A128312031394210A16A81BE5
:1023D0008B1763080317D300031362080317D20097
:1023E0000A12031365270A167A080317D50079081D
:1023F000D4007808D3007708D200AB30D900AA30D7
:10240000D8002630D7008730D6000A12031384275D
:102410000A16031CA32CC108031DDF2A061CDF2A91
:10242000C108031DDF2A061CDF2A2D08093C031CF6
:10243000372A0317D20152080A12031361200A1621
:1024400000380319372A0317D20A0313A8018B1B7C
:10245000A8178B138316031796000A12831203130F
:10246000AA210A16A81B8B1703171B2A031303178D
:10247000D60103132D080317D500D701D801D901C0
:10248000DA01DB01DC01DD01DE0101300313ED00C7
:102490005730EC001030840003175608E10055084F
:1024A000E000E8010408E7006810831B6814610E6F
:1024B000F038E300E307E23EE400323EE600610864
:1024C0000F39E407E407E607E93EE500E507E5071D
:1024D000600E0F39E507E607E50DE60DE609E60DA6
:1024E00060080F39E607E30D0730E2000A30E6071F
:1024F000E503031C772AE507E403031C7B2AE407B2
:10250000E303031C7F2AE307E203031C832A6230F0
:102510008400831707306705671384076630040259
:10252000031967170008F700031D9E2A671B9E2AE0
:10253000671AB42AE7199E2A2030A12AE7156712E4
:102540003030F707E1010408E0006110831B6114DB
:102550007708E9000A12031310250A16031760080A
:102560008400831361188317840A671F8E2ADF0192
:102570005F08073C031CDE2A57305F07840083177F
:102580000008203C0318DB2A57305F0784008317BC
:102590000008E0000313A8018B1BA8178B13031777
:1025A0006008831696000A1283120313AA210A16E2
:1025B000A81B8B170317DF0A6400B82A0313C1088E
:1025C000031D022B061C022B0317D20152080A120C
:1025D0000313B4200A1600380319022B0317D20A7A
:1025E0000313A8018B1BA8178B13831603179600E0
:1025F0000A1283120313AA210A16A81B8B170317AA
:10260000E62A0313C108031DD12B061CD12B2C086D
:10261000093C031C292B0317D20152080A12031389
:1026200061200A1600380319292B0317D20A031355
:10263000A8018B1BA8178B138316031796000A1289
:1026400083120313AA210A16A81B8B1703170D2B3D
:1026500003130317D60103132C080317D500D70162
:10266000D801D901DA01DB01DC01DD01DE01013035
:102670000313ED005730EC001030840003175608A8
:10268000E1005508E000E8010408E7006810831B3A
:102690006814610EF038E300E307E23EE400323EE6
:1026A000E60061080F39E407E407E607E93EE500C4
:1026B000E507E507600E0F39E507E607E50DE60DCE
:1026C000E609E60D60080F39E607E30D0730E20082
:1026D0000A30E607E503031C692BE507E403031C46
:1026E0006D2BE407E303031C712BE307E203031CD8
:1026F000752B6230840083170730670567138407E2
:1027000066300402031967170008F700031D902BB9
:10271000671B902B671AA62BE719902B2030932B61
:10272000E71567123030F707E1010408E000611097
:10273000831B61147708E9000A12031310250A1697
:10274000031760088400831361188317840A671FC6
:10275000802BDF015F08073C031CD02B57305F073D
:10276000840083170008203C0318CD2B57305F07E7
:10277000840083170008E0000313A8018B1BA8172F
:102780008B1303176008831696000A128312031333
:10279000AA210A16A81B8B170317DF0A6400AA2BAD
:1027A0000313C108031DF42B061CF42B0317D201DD
:1027B00052080A120313B4200A1600380319F42B26
:1027C0000317D20A0313A8018B1BA8178B138316B8
:1027D000031796000A1283120313AA210A16A81BD4
:1027E0008B170317D82B0313C108031DA32C061C3A
:1027F000A32C2B080317D60003132A080317D500B0
:10280000D701D801D901DA01DB01DC01DD01DE01EC
:1028100001300313ED005730EC0010308400031733
:102820005608E1005508E000E8010408E7006810D8
:10283000831B6814610EF038E300E307E23EE40016
:10284000323EE60061080F39E407E407E607E93E97
:10285000E500E507E507600E0F39E507E607E50D3A
:10286000E60DE609E60D60080F39E607E30D0730CF
:10287000E2000A30E607E503031C3A2CE507E4030F
:10288000031C3E2CE407E303031C422CE307E20392
:10289000031C462C623084008317073067056713DA
:1028A000840766300402031967170008F700031D48
:1028B000612C671B612C671A772CE719612C20307B
:1028C000642CE71567123030F707E1010408E000D7
:1028D0006110831B61147708E9000A1203131025A5
:1028E0000A16031760088400831361188317840A8B
:1028F000671F512CDF015F08073C031CA12C5730D8
:102900005F07840083170008203C03189E2C573073
:102910005F07840083170008E0000313A8018B1BE6
:10292000A8178B1303176008831696000A128312E8
:102930000313AA210A16A81B8B170317DF0A6400CA
:102940007B2C0313BD0163080317D3000313620834
:102950000317D2000A12031365270A16AB300317B8
:10296000D500AA30D4002630D3008730D2007A08B0
:10297000D9007908D8007808D7007708D6000A125D
:10298000031384270A16031C792D63080317D30049
:10299000031362080317D2000A12031365270A16ED
:1029A0007A080317D5007908D4007808D30077088F
:1029B000D200AB30D900AA30D8002630D7008830FA
:1029C000D6000A12031384270A16031C792D320835
:1029D000023C031DEE2C0A12C52F0A163208033CD6
:1029E000031DF52C0A12E22F0A163208043C031DBF
:1029F000FE2C0A128A1500280A168A113208053C94
:102A0000031D072D0A128A1521280A168A11320879
:102A1000063C031D102D0A128A1542280A168A1137
:102A20003208073C031D322D0317D20152080A1247
:102A30000313BA200A1600380319322D0317D20ADD
:102A40000313A8018B1BA8178B138316031796007B
:102A50000A1283120313AA210A16A81B8B17031745
:102A6000162D0313320B522D0317D20152080A12EE
:102A70000313C5200A1600380319522D0317D20A72
:102A80000313A8018B1BA8178B138316031796003B
:102A90000A1283120313AA210A16A81B8B17031705
:102AA000362D03130317D1015108043C031C782D64
:102AB000D20152080A120313D0200A160038031953
:102AC000752D0317D20A0313A8018B1BA8178B13AC
:102AD0008316031796000A1283120313AA210A16FB
:102AE000A81B8B170317592D03130317D10A542D55
:102AF000031363080317D300031362080317D200FC
:102B00000A12031365270A16AB300317D500AA3043
:102B1000D4002630D3008830D2007A08D900790852
:102B2000D8007808D7007708D6000A120313842744
:102B30000A16031CB32E63080317D300031362089D
:102B40000317D2000A12031365270A167A0803171F
:102B5000D5007908D4007808D3007708D200D901CD
:102B6000D8017A30D7008830D6000A1203138427A0
:102B70000A16031CB32E6A080317D200D4015408A6
:102B80000A12031367200A1600380319DB2D0317F6
:102B9000D40A0313A8018B1BA8178B1383160317E2
:102BA00096000A1283120313AA210A16A81B8B1778
:102BB0000317BF2D031303175208D3000310530C40
:102BC000D400D6015408D500D701D801D901DA01C3
:102BD000DB01DC01DD01DE0101300313ED005730C4
:102BE000EC001030840003175608E1005508E0009F
:102BF000E8010408E7006810831B6814610EF038D0
:102C0000E300E307E23EE400323EE60061080F39EC
:102C1000E407E407E607E93EE500E507E507600E9F
:102C20000F39E507E607E50DE60DE609E60D600854
:102C30000F39E607E30D0730E2000A30E607E50347
:102C4000031C1E2EE507E403031C222EE407E30306
:102C5000031C262EE307E203031C2A2E62308400A5
:102C6000831707306705671384076630040203196A
:102C700067170008F700031D452E671B452E671ACE
:102C80005B2EE719452E2030482EE71567123030AD
:102C9000F707E1010408E0006110831B6114770865
:102CA000E9000A12031310250A16031760088400AE
:102CB000831361188317840A671F352EDF015F08AD
:102CC000073C031C852E57305F07840083170008DC
:102CD000203C0318822E57305F07840083170008BA
:102CE000E0000313A8018B1BA8178B1303176008C0
:102CF000831696000A1283120313AA210A16A81B30
:102D00008B170317DF0A64005F2E0313A8018B1BC8
:102D1000A8178B1304308316031796000A12831228
:102D20000313AA210A16A81B8B17A8018B1BA8172F
:102D30008B1320308316031796000A128312031395
:102D4000AA210A16A81B8B17A8018B1BA8178B1387
:102D500020308316031796000A1283120313AA2148
:102D60000A16A81B8B17620BC12FE308031DC12F86
:102D70003E0BBB2EBC2EBC2F831611141118BE2E79
:102D8000D03083120317D8000A12031368240A16DE
:102D90000317D8010A12031368240A168316911424
:102DA0009118D02ED13083120317D8000A120313C2
:102DB00068240A160130F7000A1256270A16780806
:102DC0007F390317D7000130F7000A120313562783
:102DD0000A1678087F390317D6000130F7000A1267
:102DE000031356270A1678083F390317D500013018
:102DF000F7000A12031356270A1678080739B2009B
:102E00000130F7000A1256270A1678083F390317CF
:102E1000D2000130F7000A12031356270A16780869
:102E20001F390317D300F7010A12031356270A1696
:102E300078080317D40083160313111511191E2FD8
:102E400064008312031757087F3C031D2A2F0313C6
:102E5000BC2F031757080F390313B0000317570E81
:102E6000F7000F30F7057708D900DA000A30DB00E9
:102E70000A128A15031363200A168A117808B0070C
:102E8000031756080F390313AF000317560EF70048
:102E90000F30F7057708D900DA000A30DB000A1294
:102EA0008A15031363200A168A117808AF070317DF
:102EB00055080F390313AE000317550EF7000F30F6
:102EC000F7057708D900DA000A30DB000A128A1504
:102ED000031363200A168A117808AE0703175208F5
:102EE0000F390313AD000317520EF7000F30F7052B
:102EF0007708D900DA000A30DB000A128A150313BA
:102F000063200A168A117808AD07031753080F3992
:102F10000313AC000317530EF7000F30F7057708C3
:102F2000D900DA000A30DB000A128A150313632085
:102F30000A168A117808AC07031754080F390313CF
:102F4000AA00AB010317540EF7000F30F7057708FE
:102F5000D900DA000A30DB000A128A150313632055
:102F60000A168A117808AA070318AB0AD030AA07F4
:102F7000073003180830AB07BE0A3E08053C031CA7
:102F8000BE016308023C0318CE2FFF3A031DCC2F6D
:102F90006208E83C0318CE2FE301E2018A150A1209
:022FA0008A2F76
:04400E00E923FF3E65
:00000001FF
